:10A410002237B3C34EA44220436F707972696768D4
:10A42000742028632920313938332062792046721C
:10A43000616E6B2047617564652720416C6C20520A
:10A44000696768747320526573657276656421006C
:10A45000003922B0B331B0B3CDDCA51EFFCD5DB263
:10A4600032C1B532E7B53A5C00B7CA74A43D32BB1D
:10A47000B3CD56B2CDB5B23A5D00FE20C292A43A39
:10A480006500FE20C292A4213AB3115D00060BCDF7
:10A4900031B20E1A118000CD0500AF326800327C57
:10A4A000002F32BAB3115C000E11CD05003CC25A28
:10A4B000A732BAB3CD77B10D0A2B2B204E4F2046D1
:10A4C000494C4520464F554E44202B2B0D0A0A205F
:10A4D0002D2D2D3E202000CD77B1084C6F672D69C2
:10A4E0006E2064726976652F757365723A2000CDAF
:10A4F00016A53AF7B532C1B5CD5CB2CD46B23E2015
:10A50000325D003265002100002248B3CD77B10DE5
:10A510000A0A00C374A4214CB30607CDE7B1114A5F
:10A52000B30E0ACD0500CDD3B1AF32F7B53A4DB376
:10A53000FE3ACA74A5FE30DA74A5FE3AD290A5D6CA
:10A5400030FE01C262A53A4EB3FE3ACA60A5FE30A3
:10A55000DA60A5FE36D290A5D62632F7B5C374A52B
:10A560003E01473A4EB3FE3ACA70A5FE30D290A5DE
:10A570007832F7B53A16A43C473A4CB3B8D290A516
:10A580000640B8DA90A5D640325C003D32E8B5C945
:10A59000CD77B10D0A2B2B2044726976652F557348
:10A5A000657220456E747279204572726F72202B2D
:10A5B0002B070031B0B33ABAB3B7CC92B1CA92A468
:10A5C000C31AA93AE7B5CD5CB21180000E1ACD05C9
:10A5D00000CD92B12AB0B3F92A37B3C9CD86B1CD37
:10A5E00077B10D2020202020202020202020202096
:10A5F000204449534B20372E36202D204D4F4449BF
:10A600004649454420544F2052554E20494E534907
:10A630002066696C652020207C2044202D20446504
:10A640006C6574652066696C6520207C2046202D31
:10A650002046696C652073697A6520207C204A2039
:10A660002D204A756D702032322066696C65730D3D
:10A670000A2020204C202D204C6F672064726976C0
:10A68000652020207C204D202D204D617373206398
:10A690006F7079202020207C2050202D205072695E
:10A6A0006E742074657874207C2052202D205265B1
:10A6B0006E616D652066696C650D0A20202053204F
:10A6C0002D205374617420647269766520207C208B
:10A6D00054202D205461672066696C65202020205D
:10A6E000207C2055202D20556E7461672066696C92
:10A6F00065207C2056202D2056696577207465786A
:10A70000742066696C650D0A2020203F2C2F202DB7
:10A71000204D454E552020202020207C2058202DE3
:10A72000204578697420746F2064424949207C2058
:10A730003C73706163653E20616476616E6365732E
:10A7400020637572736F72202D2D20422062616329
:10A750006B732075700D0A0A00C92100B722F5B588
:10A760003D8787878787C6806F26003A5C0077EB36
:10A770002AF5B5EB060CCD31B2EB36202322F5B528
:10A780000E12115C00CD05003CC260A72AF5B5226F
:10A79000F3B522B8B3110DB7CD62B2CA52A82100E9
:10A7A000B722EFB5110D001922F1B52AF1B5EB2A48
:10A7B000EFB5E5D5060D1ABEC2C1A7231305C2B673
:10A7C000A7D1E1060DD2D3A74E1A7779122313052C
:10A7D000C2C8A72AF1B5110D001922F1B5EB2AF371
:10A7E000B5CD62B2C2ABA72AEFB5110D001922EFA9
:10A7F000B51922F1B5EB2AF3B5CD62B2C2ABA7CD44
:10A80000C8B00100002A06001100F8192BEB2AB885
:10A81000B303D511800019D1CD62B2D211A80B7843
:10A82000B1C24DA8CD77B10D0A072B2B204E4F207A
:10A830004D454D4F525920464F5220434F505920BD
:10A84000425546464552202B2B00C31AA969602267
:10A85000EDB52100B722F5B5CD77B10D0A20202046
:10A86000002AF5B57EC640CD99B13AC1B5B7CA84C4
:10A87000A8FE0ADA7FA8D60AF53E31CD99B1F1C615
:10A8800030CD99B1CD77B13A20002306087ECD991D
:10A89000B12305C28DA83E2ECD99B106037ECD9978
:10A8A000B12305C29DA87E32B3A82322F5B5CD778A
:10A8B000B1203A20003A45B3B7CA27A9CDB9B1FEB5
:10A8C00020CA0EAAFE0DCA0EAAFE42CA27AAFE433D
:10A8D000CAB4ADFE44CA8EAAFE46CA6BA9FE4ACAD5
:10A8E00007AAFE4CCAD7A4FE4DCA82ADFE50CAA329
:10A8F000ACFE52CA33ABFE53CA56AAFE54CA51A983
:10A90000FE55CA3BA9FE56CA49ACFE58CAC3A5FEAD
:10A910001BCAC3A5CDDCA5CDB5B22AF5B511F3FF91
:10A920001922F5B5C358A83AE5B53C32E5B5FE168F
:10A93000C20EAA3EFF3245B3C3BCA8AF321DB62A31
:10A94000F5B511FFFF197EFE2A3620CA6FA9C30E86
:10A95000AA2AF5B511FFFF197EFE2ACA0EAA362AC9
:10A960003EFF321DB632E4B5C36FA9AF32E4B53E47
:10A9700008CD99B1CD25B20E2311F8B5CD05002A29
:10A9800019B622E9B52100002219B63AB4B3F56F21
:10A99000EB2AE9B5190604CD68B2F10F0F0FE61FD7
:10A9A0002FA56F3AE4B5B7CACAA9EB3A1DB6B7CA24
:10A9B000BDA92A48B3192248B3EBC3CAA92A48B390
:10A9C0007D936F7C9A672248B3EBCD98B23E099095
:10A9D000321CB6CD74B2CD77B16B003AE4B5B7CACC
:10A9E0000EAA2A48B3CD98B23A1CB690473E20CD65
:10A9F00099B105C2EFA93E28CD99B1CD74B2CD77FA
:10AA0000B16B2900C30EAAAF3245B332E5B52AF5C2
:10AA1000B5EB2AF3B5CD62B2C258A8CD92B12100F0
:10AA2000B722F5B5C358A82AF5B5110DB7CD62B256
:10AA3000C240AACD92B12AF3B5110D001922F5B585
:10AA4000CD77B10D0A3C2D20002AF5B511E6FF198E
:10AA500022F5B5C361A8CD77B1746F7261676520C7
:10AA600072656D61696E696E67206F6E20647269D0
:10AA700076653A2000CD16A5CD46B2CD77B10D0A48
:10AA80000A00CDB5B23ABBB3CD56B2C31AA9CD2593
:10AA9000B2CD77B1656C6574653F2028592F4E297A
:10AAA0003A2000CDB9B1FE59C21AA911F8B50E135A
:10AAB000CD05003CC2D3AACD77B10D0A2B2B204E79
:10AAC0004F2046494C4520464F554E44202B2B00E5
:10AAD000C31AA92AF5B5E511F3FF1922F5B5EBE183
:10AAE000EBE52AF3B5CD62B2E1EBCAF5AA060DCDCE
:10AAF00031B2C3E0AAEB22F3B51100B7CD62B2C206
:10AB00000EAA2AF5B5CD62B2C20EAACD77B10D0A52
:10AB10000A202020202B2B204C69737420456D7057
:10AB20007479202B2B0D0A0A202D2D2D3E2020007C
:10AB3000C3D7A42AF5B511F3FF1911C2B5060CCD80
:10AB400031B2CD77B1656E616D652066696C652047
:10AB5000746F3A2000114AB30E0ACD0500CDD3B16F
:10AB600021D2B5360023E5060BCDE7B1E1EB214B51
:10AB7000B34E23EBCDEFB1E5692600193620E1068F
:10AB800008CDFBB1DAB3A5FE20CAC8ABFE2ECAA71A
:10AB9000AB772305C281ABCDFBB1DAC8ABFE20CACF
:10ABA000C8ABFE2EC297AB060321DBB5CDFBB1DAF5
:10ABB000C2ABFE20CAC2ABFE2ECAC2AB772305C20F
:10ABC000ACAB21DEB5CD3CB211C3B521D3B50E0B74
:10ABD0001AE680473E7FA6B07723130DC2D0AB3A6A
:10ABE000C2B532F8B5060B21D3B511F9B5CD31B2E6
:10ABF0002104B6CD3CB211F8B50E11CD05003CCA0A
:10AC00002AACCD77B10D0A2B2B2046494C4520416B
:10AC10004C524541445920455849535453202B2BFD
:10AC20000D0A0720202000C31AA92AF5B511F4FF48
:10AC300019EB21D3B5060BCD31B211C2B50E17CD2C
:10AC400005003CC21AA9C3B7AACD77B10D0A3C438F
:10AC500054524C2D583E2063616E63656C732C20FA
:10AC60003C73706163653E207475726E73207570FD
:10AC7000206F6E65206C696E652C206F746865723C
:10AC8000206B6579732070616765207363726565F9
:10AC90006E2E0D0A0A003E0132E6B5321EB63E02A5
:10ACA000C3B2ACAF321EB63E05C3B2ACAF321EB6B5
:10ACB0003E0432BCB3CD25B21180000E1ACD050082
:10ACC0002104B6CD3CB211F8B50E0FCD05003CC243
:10ACD000F2ACCD77B12B2B20554E41424C45205440
:10ACE0004F204F50454E2046494C45202B2B00C34A
:10ACF0001AA9AF3218B611F8B50E14CD0500B7C2B7
:10AD00001AA921800006807EE67FFE1ACA1AA95F72
:10AD1000C5E5D53ABCB34FCD05003A1EB6B7D1C490
:10AD200035AD0E0BCD0500E1C1B7C21AA92305C28E
:10AD300007ADC3F6AC7BFE0AC03AE6B53C32E6B5D9
:10AD4000FE16D8AF32E6B5CD77B120205B6D6F72BD
:10AD5000652E2E2E5D0D00CDC7B1FE20F5CD77B14D
:10AD600020202020202020202020200D00F1C2774C
:10AD7000AD3E1532E6B5C9FE1BCAB3A5FE18CAB36F
:10AD8000A5C9210CB722F5B53E2ABE2322F5B5CAC6
:10AD9000B0AD2AF5B5EB2AF3B5CD62B2CAA5AD2A9E
:10ADA000F5B5C388ADAF3246B32F3247B3C352A80F
:10ADB000AF3247B321000022BDB5CD25B22104B684
:10ADC000CD3CB2AF3218B6062021F9B511C3B5CDCE
:10ADD00031B211F8B50E0FCD05003CC202AECD77F1
:10ADE000B10D0A2B2B20554E41424C4520544F208B
:10ADF0004F50454E20534F55524345202B2B00C3F7
:10AE00001AA93A46B3B7C274AECD77B108436F7092
:10AE10007920746F2064726976652F757365723A54
:10AE20002000CD16A53A5C00473AF8B5B8C271AE1D
:10AE30003AF7B5473AC1B5B8C271AECD77B10D0A90
:10AE4000072B2B20447269766573206F722055732F
:10AE50006572204172656173206D7573742062653F
:10AE600020646966666572656E74202B2B00C31AB8
:10AE7000A9CD46B23A5C0032C2B53AF7B5CD5CB264
:10AE80003A47B3B7CACBAE11C2B50E11CD05003CDF
:10AE9000CAD3AECD77B10D0A202D2D2D3E20436FA4
:10AEA0007079206578697374732C2065726173659D
:10AEB0003F2028592F4E293A2000CDB9B1FE59CA5A
:10AEC000CBAE3AC1B5CD5CB2C30EAA11C2B50E135A
:10AED000CD050011C2B50E16CD05003CC208AFCDA0
:10AEE00077B10D0A2B2B2044657374696E61746908
:10AEF0006F6E204469726563746F72792046756C59
:10AF00006C202B2B00C31AA9060821C3B5113CAF36
:10AF1000CD31B2130603CD31B23A46B3B73E0ACCB7
:10AF200099B1CDA8B1CD77B10D202D2D2D3E204367
:10AF30006F7079696E672066696C6520202020201B
:10AF4000202020202E2020202000AF32E3B53AC15F
:10AF5000B5CD5CB221000022EBB52AB8B322B6B35E
:10AF60002AB6B3EB0E1ACD050011F8B50E14CD05B7
:10AF700000B7CA9AAF3DCAC6AFCD77B10D0A2B2B29
:10AF800020534F555243452052454144204552528B
:10AF90004F52202B2B0700C31AA92AB6B306807E76
:10AFA000CDF3B02305C29FAF2AB6B311800019229A
:10AFB000B6B32AEBB52322EBB5EB2AEDB5CD62B2E1
:10AFC000C260AFC3CBAF3EFF32E3B53AF7B5CD5C5D
:10AFD000B22AB8B322B6B32AEBB57CB5CA2BB02BD4
:10AFE00022EBB52AB6B3E5EB0E1ACD0500E11180D0
:10AFF000001922B6B311C2B50E15CD0500B7CAD7D8
:10B00000AFCD77B10D0A2B2B20434F505920444927
:10B01000534B2046554C4C202B2B070011C2B50E2C
:10B0200013CD0500AF3246B3C31AA93AE3B5B7CA88
:10B030004EAF11C2B50E10CD05003CC25EB0CD774B
:10B04000B10D0A2B2B20434F505920434C4F5345F1
:10B05000204552524F52202B2B0700C31CB02ABD53
:10B06000B522BFB521000022BDB51180000E1ACD5A
:10B07000050021CEB5CD3CB211C2B50E0FCD0500F5
:10B080003CCA53B1AF32E2B511C2B50E14CD0500C2
:10B09000B7CAB7B03DCA0DB1CD77B10D0A2B2B2081
:10B0A000434F50592052454144204552524F52205F
:10B0B0002B2B0700C31AA921800006807ECDF3B098
:10B0C0002305C2BCB0C388B021BDB30E00EB210084
:10B0D0000079C50608AC6729D2E3B03E10AC673EE4
:10B0E00021AD6F05C2D7B0C1EB72247325230CC20A
:10B0F000CDB0C9C5E52ABDB5EB0600AA4F21BDB349
:10B10000097EAB57245EEB22BDB5E1C1C93AC1B59A
:10B11000CD5CB22ABDB5EB2ABFB5CD62B2C253B188
:10B12000CD77B10D202D2D2D3E20436F707920431A
:10B13000524320766572696669656420202020206C
:10B1400020202020003A47B3B7C20EAA2F3246B3C0
:10B15000C392ADCD77B10D0A072B2B204572726FCC
:10B1600072206F6E2043524320636F6D7061726571
:10B17000202B2B00C30EAAE37EE67FCD99B1237E60
:10B18000B7C278B1E3C906113E0ACD99B105C288AC
:10B19000B1C93E0DCD99B13E0AF5C5D5E55F0E02A8
:10B1A000CD0500E1D1C1F1C93E0DCD99B1061E3EDC
:10B1B00020CD99B105C2B1B1C90E01CD0500FE6126
:10B1C000D8FE7BD0E65FC90E061EFFCD0500B7CACC
:10B1D000C7B1C9214BB34678B7CAB3A5237ECDBE4C
:10B1E000B17705C2DCB1C936202305C2E7B1C91A5F
:10B1F000FE20C0130DCAB3A5C3EFB11A13FE20D8A9
:10B20000E5C5FE5BD219B20608211DB2BECA19B24D
:10B210002305C20CB2B7C1E1C9C1E137C92A2C3A32
:10B220003B3C3D3E3F2AF5B511F3FF1911F8B50639
:10B230000C7EE67F12231305C231B2C90604360024
:10B240002305C23EB2C90E19CD050032BBB30E0DA7
:10B25000CD05003AE8B55F0E0EC305005F0E20C3B2
:10B2600005007ABCC07BBDC905C87CB71F677D1FC0
:10B270006FC368B2F5C5D5E501F6FF11FFFF0913ED
:10B28000DA7EB2010A0009EB7CB5C474B27BC63029
:10B29000CD99B1E1D1C1F1C9110900CD62B2060168
:10B2A000D01E63CD62B20602D011E703CD62B206B2
:10B2B00003D00604C90E19CD05003C325C00C6401F
:10B2C000322FB30E1FCD050023237E32B5B3237E6C
:10B2D00032B4B323235E2356EB22B2B30E1BCD054B
:10B2E00000EB2AB2B323010000D51A1E0817DAF2C8
:10B2F000B203572B7DB4CA03B37A1DC2EDB2D1138A
:10B30000C3E9B2D169603AB5B3D603CA13B3293DD4
:10B31000C20EB3CD74B2CD77B16B20627974657310
:10B320002066726565206F6E2064726976652020E4
:10B330003A0D0A202020000000C93F3F3F3F3F3F19
:0CB340003F3F3F3F3FFF00FF00002000A8
:00A410004C
